:100000000C948E050C94D5050C94D5050C94D5054F
:100010000C94D5050C94D5050C94D5050C94D505F8
:100020000C94D5050C94D5050C947C2B0C944E2C7B
:100030000C94C0210C94D5050C94D5050C94D505D1
:100040000C94D5050C94D5050C94D5050C94D505C8
:100050000C94D5050C9428220C94D5050C94D50548
:100060000C94D5050C94D5050C94D5050C94D505A8
:100070000C94D5050C94D5050C94D5050C94D50598
:100080000C94D5050C94D5050C94D5050C94D50588
:100090000C94D5050C94D5050C94D5050C94D50578
:1000A0000C94D5050C94D5050C94D505F607FB07E3
:1000B0000508F907FE0703080108910893089E0840
:1000C0009508970899089B089D08A008A208A4080D
:1000D000AF08A608A808AA08AC08AE08B1087D17A2
:1000E0007D17B717B717EC170C187919B5194E18F3
:1000F000B519FE18FE187119B519B519B0190B19F3
:100100000B190B190B190B190B190B190B190B19CF
:100110000B190B190B190B190B190B190B191D19AD
:100120002A19311938194219401A401A521A521A0A
:10013000491A521A521A521A401A401A4E1A521A90
:10014000521A4E1ABB2CDD2CCB2DDD2CCB2D222DA3
:10015000452DCB2D9A2DAD2D6572676F646F782F6D
:100160006572676F646F785F657A5F3239343061CA
:100170006564346137383363346132666633322004
:100180004020302E352E3438006572676F646F78EA
:100190002F6572676F646F785F657A5F32393430CC
:1001A0006165643461373833633461326666333293
:1001B000204020302E352E3438000000F0A12900D8
:1001C0002B002A61E100006700001E0014000400FB
:1001D0001D005200E3001F001A0016001B00510012
:1001E0002B00200008000700060050002C00210012
:1001F0001500090019004F000653220017000A00DD
:100200000500000002544C0001540000045300009B
:1002100003542A0001540000045300000354230037
:100220001C000B00110000000254240018000D00F7
:1002300010005200065325000C000E00360051003D
:100240002C00260012000F00370050002800270065
:100250001300334538004F0029002D0031003400D1
:10026000E5000067000010500100010001000100DE
:1002700000003A002E0057005600010001003B002C
:10028000230225023800010001003C002F02260253
:100290002F00010001003D00300227023000010064
:1002A00001003E003102350035020000010001006E
:1002B0000100000001000000010001000100000039
:1002C0000100000001003F001E023602240200006F
:1002D000010040001F02370233000100010041000D
:1002E00020022D02360001000100420021023302EB
:1002F000630001000100430022021450310001009C
:1003000010504400450034020100010000000100CB
:100310002B012A01E101E20100001E011401040188
:100320001D01520101001F011A0116011B0151019B
:100330002B012001080107010601500101002101E4
:100340001501090119014F010100220117010A01DC
:100350000501000001004C01010000000100000047
:1003600001002A010100000001000000010023013A
:100370001C020B01110100000100240118010D01F4
:1003800010015201010025010C010E01360151013D
:100390000100260112010F01370150012801270138
:1003A0001301330138014F01010001000100010078
:1003B000E101E2010000010001002A04E104E0047F
:1003C00000001E04140404041D04520401001F0450
:1003D0001A0416041B0451042B0420040804070407
:1003E000060450042C0421041504090419044F04C4
:1003F0000100220417040A040504000001004C0453
:10040000010000000100000001002A0401000000BA
:1004100001000000010023041C040B04110400006F
:100420000100240418040D041004520401002504E2
:100430000C040E04360451042C04260412040F0488
:1004400037045004280427041304330438044F04E9
:100450000100010001000100E104E004000010506F
:1004600001002A0001000100000001002E005700D9
:100470002D005200010001002302550038005100F8
:100480002B0001002F0226022F0050002C0001003B
:100490003002270230004F0001000100010001007E
:1004A0000100000001004C000100000001000000FC
:1004B00001002A000100000001000000010001000D
:1004C00001000100010000000100010024002100E2
:1004D0001E00520001000100250022001F005100F3
:1004E0002C000100260023002000500028000100FD
:1004F0002700270027004F001050010001000100D5
:100500000100010000001050010001000100005C2A
:10051000000001000100F2000100010001000100E3
:10052000F000F10001000100F50001000100F300FE
:1005300001000100F4000100FF00FD00FF000100C8
:1005400001000100010001000100000001000100A4
:100550000100000001000000010001000100000096
:100560000100000001000100010001000100000085
:100570000100010001000100010001000100010073
:100580000100010001000100010001000100010063
:1005900001000100580001000100010001000100FC
:1005A0001050010001000100010001000000105086
:1005B0002B0201000100E00600001E0214020402EA
:1005C0001D02010001001F021A0216021B02010097
:1005D0002B0220020802070206020100010021028C
:1005E00015020902190201000100220217020A0283
:1005F00005020000E002010001000000010000000F
:10060000E20201000100000001000000E2022302FA
:100610001C020B0211020000E002250218020D026A
:1006200010020100010026020C020E023602010037
:100630000100270212020F023702010028022D02D8
:1006400013023302380201001050010001000100C2
:100650000100E006000000000000000000002A2B5E
:100660002800000000000000000000000000000062
:100670000029000000002C1E3420212224342627CB
:10068000252E362D3738271E1F20212223242526EC
:100690003333362E37381F0405060708090A0B0CBA
:1006A0000D0E0F101112131415161718191A1B1C02
:1006B0001D2F3130232D350405060708090A0B0CC0
:1006C0000D0E0F101112131415161718191A1B1CE2
:1006D0001D2F3130354C00000000000000000000EC
:1006E000000000000000000000000000000000000A
:1006F00000000000000000010101010101000101F2
:1007000001010000000000000000000000000000E7
:1007100001000100010101010101010101010101CB
:1007200001010101010101010101010101010101B9
:1007300001000000010100000000000000000000B6
:1007400000000000000000000000000000000000A9
:100750000001010101006801F000B40078005A00B6
:10076000643214643214783C1E1E140A0500000022
:10077000000101010202030405050607090A0B0C2A
:100780000E0F1112141517191B1D1F212325282ABE
:100790002C2F313436393B3E414346494C4F52555C
:1007A000585A5D6164676A6D707376797C7F838661
:1007B000898C8F9295989B9EA2A5A7AAADB0B3B63F
:1007C000B9BCBEC1C4C6C9CBCED0D3D5D7DADCDE66
:1007D000E0E2E4E6E8EAEBEDEEF0F1F3F4F5F6F84A
:1007E000F9FAFAFBFCFDFDFEFEFEFFFFFFFFFFFF37
:1007F000FFFEFEFEFDFDFCFBFAFAF9F8F6F5F4F358
:10080000F1F0EEEDEBEAE8E6E4E2E0DEDCDAD7D5A3
:10081000D3D0CECBC9C6C4C1BEBCB9B6B3B0ADAAE5
:10082000A7A5A29E9B9895928F8C898683807C79C0
:100830007673706D6A6764615D5A5855524F4C49C2
:100840004643413E3B393634312F2C2A282523217B
:100850001F1D1B1917151412110F0E0C0B0A090777
:10086000060505040302020101010000000000006A
:100870000000010101010101010101020202020265
:100880000202020203030303030303030404040438
:1008900004040505050505060606060607070707FD
:1008A000080808080909090A0A0A0A0B0B0B0C0CAC
:1008B0000C0D0D0D0E0E0F0F0F1010111111121245
:1008C00013131414151516161717181819191A1AC0
:1008D0001B1C1C1D1D1E1F1F20202122222324251E
:1008E0002526272728292A2B2B2C2D2E2F2F303158
:1008F0003233343536363738393A3B3C3D3E3F406B
:1009000041424344464748494A4B4C4D4F5051524F
:1009100053555657585A5B5C5E5F60626364666706
:10092000696A6C6D6E707173747678797B7C7E8089
:1009300081838486888A8B8D8F91929496989A9BD6
:100940009D9FA1A3A5A7A9ABADAFB1B3B5B7B9BBE7
:10095000BDBFC1C4C6C8CACCCFD1D3D6D8DADCDFBC
:10096000E1E4E6E8EBEDF0F2F5F7FAFCFF160345FB
:1009700000720067006F0044006F0078002000459F
:10098000005A00000016034500720067006F004423
:10099000006F007800200045005A000000040309A1
:1009A0000409026D00040100A0FA0904000001031B
:1009B0000101000921110100012240000705810306
:1009C00008000A09040100010301020009211101C4
:1009D0000001224D000705820308000A09040200F5
:1009E0000103000000092111010001223600070562
:1009F000830308000A090403000103000000092121
:100A000011010001223900070584032000011201B1
:100A1000100100000008EDFE0713010001020001B3
:100A200005010906A101050719E029E715002501BF
:100A300095087501810205081901290595057501BB
:100A400091029501750391010507190029F7150019
:100A5000250195F875018102C005010980A1018574
:100A6000021601002603001A81002A8300751095E2
:100A7000018100C0050C0901A101850316010026B2
:100A80009C021A01002A9C02751095018100C00584
:100A9000010902A1010901A1000509190129051592
:100AA00000250195057501810295017503810105F8
:100AB00001093009311581257F95027508810609E4
:100AC000381581257F950175088106050C0A3802C5
:100AD0001581257F950175088106C0C005010906AD
:100AE000A101050719E029E7150025019508750101
:100AF00081029501750881010508190129059505EF
:100B0000750191029501750391010507190029FFEF
:100B1000150026FF00950675088100C011241FBE30
:100B2000CFEFDAE0DEBFCDBF04B603FE27C0809171
:100B3000B7039091B803A091B903B091BA0387307D
:100B4000904BA740B04BD1F41092B7031092B8036A
:100B50001092B9031092BA0314BE84B7877F84BF82
:100B60000FB6F894A895809160008861809360002A
:100B7000109260000FBEE0E0FFE3099511E0A0E0F5
:100B8000B1E0E0E5FFE502C005900D92AA3DB10796
:100B9000D9F723E0AAEDB1E001C01D92A73BB2074F
:100BA000E1F70E94A9280C94A62F0C940000109243
:100BB000B9008AE08093B800089594EA9093BC004D
:100BC0009091BC0097FFFCCF9091B900987F98302E
:100BD00021F0903111F081E008958093BB0084E80A
:100BE0008093BC008091BC0087FFFCCF8091B9004E
:100BF000887F883111F0803471F780E0089584E9AE
:100C00008093BC008091BC0084FDFCCF089580934C
:100C1000BB0084E88093BC008091BC0087FFFCCFC0
:100C20009091B900987F81E0983209F480E00895AE
:100C300084E88093BC008091BC0087FFFCCF80914A
:100C4000BB00089580B38C7080BB81B3836F81BB80
:100C5000089580910001811115C080E40E94DD0596
:100C60008093000181110CC082E10E9407068093ED
:100C70000001811105C08FEF0E94070680930001DB
:100C80000E94FF0584B1807F84B985B1807F85B9DA
:100C90008AB1837F8AB98BB1837F8BB93E9846989E
:100CA000089508950C94DA070E94DB0C80930001EC
:100CB0000E9429060E9422062BED31E0EFE2F2E0CD
:100CC0004EE04E0F119280E090E0D901A80FB91FBD
:100CD0001C92019686309105C1F72A5F3F4F4E1353
:100CE000F1CF0C94E1090E94DB0C809300010E947B
:100CF00029060E942206EFE2F2E08EE08E0F1192AA
:100D00008E13FDCF089526E0829FC0011124FC01BF
:100D1000E552FE4F20E030E080E041E050E090817D
:100D2000992319F09150908307C0BA01022E01C097
:100D3000660F0A94EAF7862B2F5F3F4F31962630D5
:100D4000310569F7089596E0699FB001112420E00C
:100D500030E090E04FE0FC01022E02C0F595E795EF
:100D60000A94E2F7E0FF06C0F901E60FF71FE5522B
:100D7000FE4F40832F5F3F4F2630310561F70895C6
:100D8000AF92BF92CF92DF92EF92FF920F931F9399
:100D9000CF93DF9380910001882379F08091DA016D
:100DA0008F5F8093DA01811108C00E94DB0C809371
:100DB0000001811102C00E946D0C8FE2E82E82E0DA
:100DC000F82E00E010E0CC24C394D12CAA24A394E4
:100DD000C02F0730110500F58091000181113CC042
:100DE00080E40E94DD0580930001811112C082E140
:100DF0000E9407068093000181110BC0C601002EDE
:100E000001C0880F0A94EAF780950E940706809334
:100E100000010E94FF0520C00A30A1F028F408302C
:100E200059F0093061F005C00C3089F070F00D30D8
:100E300089F0209A289810C0219A29980DC0229AEA
:100E40002A980AC0239A2B9807C0529A01C0539A35
:100E50005B9802C03E9A469880EA8A95F1F78C2FFB
:100E60000E948306D82F0730110518F580910001E4
:100E7000811144C080E40E94DD0580930001882335
:100E800011F0B12C12C083E10E940706809300018B
:100E90008111F7CF81E40E94DD058093000181116B
:100EA000F0CF0E941806B82EB0940E94FF059B2D2B
:100EB00026C08FB181708A25799902C092E001C065
:100EC00090E0892B7C9902C094E001C090E0982BBF
:100ED0007D9902C038E001C030E0932B7E9902C0BA
:100EE00020E101C020E0922B2FB12095221F222764
:100EF000221F2295220F207E922B01C090E0F70145
:100F000080819D23D095D823D92B6C2F8D270E94CB
:100F1000A306F701D1937F010E9429060F5F1F4F9F
:100F20000E30110509F054CF0E94E30981E0DF91F2
:100F3000CF911F910F91FF90EF90DF90CF90BF90D6
:100F4000AF900895E82FF0E0E15DFD4F80810895B6
:100F50000895611108C0FC018281882321F089E88D
:100F600091E00E94B60980E090E00895FB018E3C7C
:100F70002CE5920769F08F3C2CE5920789F08D3CB7
:100F80009C45B1F482818823A1F00E943C210EC0CF
:100F90008281882371F088E591E00E94B60906C03D
:100FA0008281882331F081E00E943C1180E0089525
:100FB00081E008956091FF02709100038091010328
:100FC000909102030E94EC2056985E9825982D98E7
:100FD00026982E9827982F9890E0FC013197E730BB
:100FE000F105A8F4EA5AFF4F0C94582F259A2D9A30
:100FF0000895259A2D9A269A2E9A0895259A2D9A23
:1010000004C0259A2D9A269A2E9A279A2F9A0895E7
:1010100081E008950C94B6070E942E1A2FEF84E306
:101020009CE0215080409040E1F700C000000C940B
:101030004E22FF920F931F93CF93DF938C01FC01FD
:10104000C081D18180918E02811113C08281882359
:1010500049F0CE010E944F1FF82E682FCE010E944A
:10106000F21E04C0CE010E94221FF82EBE018F2D59
:1010700004C0CE010E944F1FBE010E94F809EC017E
:10108000B8010E940A08882309F469C1B801CE0199
:101090000E941E0C882309F462C1B801CE010E948F
:1010A0002A0D882309F45BC1C13CFCE5DF0741F44C
:1010B000F8018281882309F452C10E94C4104FC1F3
:1010C000C23C8CE5D80708F0A6C0C5319CE5D9071D
:1010D00008F07EC0C230ECE5DE0708F452C0F8012B
:1010E0008281882309F459C00E945D21811102C0C8
:1010F0000E943C210E94702190E09093A90380936C
:10110000A803FE01E350FC45E231F10530F4E35A57
:10111000FF4F8091A8030C94582F8091A803816001
:1011200027C0826025C0846023C0806121C08062A6
:101130001FC080641DC080681BC08460886018C0A8
:101140008E7F16C08D7F14C08B7F12C08F7E10C023
:101150008F7D0EC08F7B0CC08F770AC08B7F877FFF
:1011600007C087FB222720F991E0922790FB87F99F
:101170008093A8038091A8030E9474210E942E1AD4
:10118000EEC0C115FCE5DF0781F0C130DC45A9F0F8
:1011900081E08093410280934202C801DF91CF91A8
:1011A0001F910F91FF900C940808F8018281882309
:1011B00009F4D5C00E940C08D2C0F80182818823AE
:1011C00009F4CDC080912C03816080932C03C7C0AB
:1011D000CF3B9CE5D90741F4F8018281882309F4CB
:1011E000BEC00E94B711BBC0C03CECE5DE0740F0BA
:1011F000F8018281882309F4B2C00E94AC10AFC00C
:10120000CE3BDC4529F6F8018281882309F4A7C08A
:101210000E94C111A4C0C53C8CE5D80741F4F80177
:101220008281882309F49BC00E94221198C0C63C89
:101230009CE5D907D8F4F8018281C33CFCE5DF07BF
:1012400031F4882309F48BC00E94F51088C0C43C97
:10125000DC4530F4882309F482C00E94E3107FC08B
:10126000882309F47CC00E94071179C0C73CECE5D3
:10127000DE0781F5F8018281882361F01092420235
:101280000E94F2219093400280933F0280E20E94EC
:10129000321765C00E94732081FF05C081E08093F2
:1012A0004102809342028091420281110FC08091DD
:1012B0003F02909140020E94FE21883C910530F44B
:1012C00087E20E94101687E20E94E31680E20E94E5
:1012D000391745C0C73CFCE5DF0760F5F80182819E
:1012E000882351F0109241020E94F22190933E0215
:1012F00080933D0282E0CBCF0E94732085FF05C022
:1013000081E08093410280934202809141028111E9
:101310000FC080913D0290913E020E94FE21883CC8
:10132000910530F486E20E94101686E20E94E316D0
:1013300082E0CDCFCA3C8CE5D80731F4F801828138
:10134000882369F080E009C0CB3CDC4509F020CF60
:10135000F8018281882319F082E00E943F2980E011
:10136000DF91CF911F910F91FF9008950F931F93DD
:10137000CF938C01F80124912223F9F030E0F90198
:10138000EA5AF94FC491F901EA52F94F2491222304
:1013900059F081EE0E9410168C2F0E9410168C2F8F
:1013A0000E94E31681EE04C08C2F0E9410168C2F31
:1013B0000E94E3160F5F1F4FDDCFCF911F910F915A
:1013C00008950C94C50C0C945206282F882339F0EC
:1013D00090E02A3010F44D9608950697089587E21C
:1013E00090E0089508950C94F2090C94F30908957F
:1013F00096E0799FF001112494E5899FE00DF11D9D
:101400001124E60FF11DEE0FFF1FE254FE4F8591F0
:1014100094910895880F991FFC01E654FE4F859121
:10142000949108950E94F8090E94A00B811520E470
:101430009207B0F5811540E3940708F0DBC0803EC9
:101440009105D8F4803C910508F069C0883A91056F
:1014500078F4853A910508F065C08130910509F46A
:101460006EC108F425C18430910508F068C120C11F
:101470008D3B910508F461C01BC18F3F910509F0B8
:1014800048F4803F910508F0AFC0883E910508F40C
:1014900056C10EC1811560E2960708F0A7C00895F5
:1014A000811574E59707D8F4811523E5920708F0B4
:1014B000DDC0811541E5940740F4811560E596078C
:1014C00008F0A2C09F70906A0895811572E5970791
:1014D00008F0B6C0982F8827816F906A089581150B
:1014E00026E5920750F4811545E5940708F0D4C02D
:1014F000982F8827846F906A0895811568E596076C
:1015000008F4D6C0811579E5970708F4CAC09C0194
:1015100030562115304208F0CBC09F71C7C0805CA7
:10152000910965C0853A910509F4C5C0863A9105CF
:1015300009F0C4C082E890E40895883A910509F45E
:10154000C0C0893A910509F4BFC08A3A910509F4EF
:10155000BEC08B3A910509F4BDC08C3A910509F4DF
:10156000BCC08B3B910509F4BBC08C3B910509F4D1
:10157000BAC08D3A910509F4B9C0803B910509F4D0
:10158000B8C08E3A910509F4B7C08F3A910509F4B5
:10159000B6C0813B910509F4B5C0823B910509F4C1
:1015A000B4C0833B910509F4B3C0843B910509F4B1
:1015B000B2C0853B910509F4B1C0863B910509F4A1
:1015C000B0C0873B910509F4AFC0883B910509F491
:1015D000AEC0893B910509F4ADC08A3B910509F481
:1015E000ACC080E094E40895906508959F700E94D7
:1015F0000A0A08959C01332793FF03C0C901986C20
:101600000895C901906C0895482F437021E030E09F
:1016100002C0220F331F4A95E2F73C68AC0164E038
:10162000569547956A95E1F74370342B8F708695F0
:10163000869560E2869FC0011124822B932B08952A
:10164000482F4695469570E2479FA001112483706C
:10165000992721E030E0B90102C0660F771F8A9513
:10166000E2F7CB01842B952B9C680895482F469573
:10167000469570E2479FA00111248370992721E0CD
:1016800030E0B90102C0660F771F8A95E2F7CB01FF
:10169000842B952B9A6808958F719927982F882706
:1016A00005C0982F8827806F906A089590620895EA
:1016B00080E090E0089581E890E4089583E890E464
:1016C000089582EE94E4089589EE94E408958AEEF4
:1016D00094E4089585EB94E4089586EB94E40895EA
:1016E00083EB94E4089584EB94E4089587EB94E409
:1016F00008958CEC94E408958DEC94E4089583E8C7
:1017000095E408958AE895E4089582E995E40895BA
:1017100084E995E4089581E296E4089583E296E4ED
:10172000089584E296E4089585E296E4089586E2B9
:1017300096E4089587E296E408958AE296E408958F
:101740008238910549F1B0F48133910509F458C00C
:1017500048F48932910509F44EC08A32910509F4A2
:1017600054C008958533910509F440C0893391052B
:1017700099F00895833E910529F138F4803E910552
:1017800091F0823E9105A1F00895863E9105F9F011
:10179000873E910531F108952091A80320FD3AC0BC
:1017A00021FD38C008958091A80380FD35C032C066
:1017B0008091A80382FF32C08091A80384FD30C0CD
:1017C00083EE39C08091A80382FD28C0F5CF8091B7
:1017D000A80383FF27C08091A80384FD21C087EE62
:1017E0002AC08091A80383FD1DC0F5CF8091A80376
:1017F00085FD1AC01BC08091A80385FD17C014C0C9
:101800008091A80386FD14C015C08091A80386FDB1
:1018100011C00EC080EE0FC089E30DC082EE0BC078
:1018200080E009C086EE07C089E205C085E303C0F9
:101830008AE201C081E390E0089508950F931F9319
:10184000CF93FB012281211102C0C1E041C08C0174
:10185000C0915002C11125C085319C45B1F70E944D
:101860001D0C81E0809350020E94F22190934F0260
:1018700080934E021092430210924502109244024D
:1018800010924702109246021092490210924802AA
:1018900010924B0210924A0210924D0210924C028A
:1018A00017C080914E0290914F020E94FE21883C09
:1018B000910558F690914302E92FF0E0EE0FFF1FDB
:1018C000EC5BFD4F118300839F5F90934302C0E068
:1018D0008C2FCF911F910F91089556985E9825985F
:1018E0002D9826982E9827982F988FEF90E0909318
:1018F00089008093880090938B0080938A00909356
:101900008D0080938C00259A2D9A2FEF80E792E02E
:10191000215080409040E1F700C00000269A2E9AA6
:101920002FEF80E792E0215080409040E1F700C027
:101930000000279A2F9A2FEF80E792E021508040F5
:101940009040E1F700C0000025982D982FEF80E728
:1019500092E0215080409040E1F700C000002698BE
:101960002E982FEF80E792E0215080409040E1F7E1
:1019700000C0000027982F9856985E9825982D98BB
:1019800026982E9827982F98089589EA80938000AA
:1019900089E08093810024982C983F988AB18F7CAD
:1019A0008AB96E98479A8BB180638BB9769A0E94F8
:1019B0006D0C0C94510680E28093000180915102DD
:1019C00081110EC00E94D70581E0809351022FEF54
:1019D00083ED90E3215080409040E1F700C000008B
:1019E00080E40E94DD058093000181112EC00E94D9
:1019F000070680930001811128C00E94070680938A
:101A00000001811122C08FE30E940706809300012C
:101A100081111BC00E94FF0580E40E94DD058093B8
:101A20000001811112C08CE00E9407068093000122
:101A300081110BC00E94070680930001811105C02F
:101A40008FE30E940706809300010E94FF058091AA
:101A500000010895CF93DF93813020E89207D0F002
:101A6000FB0122812223B1F0EC018091520281110D
:101A700009C08CE090E00E945E2F0E944E0D81E034
:101A8000809352020E94550DCE019F770E94130E43
:101A90000E94CB0D81E0DF91CF9108958093530296
:101AA000682F8CE090E00C94722FE0910201F0918D
:101AB0000301808180935D0381FF03C081EE0E945A
:101AC000E31680915D0385FF03C085EE0E94E31657
:101AD00080915D0380FF03C080EE0E94E316809139
:101AE0005D0384FF03C084EE0E94E31680915D03D2
:101AF00082FF03C082EE0E94E31680915D0386FFA1
:101B000003C086EE0E94E31680915D0383FF03C04D
:101B100083EE0E94E31680915D0387FF03C087EE8A
:101B20000E94E316809153028130A1F078F0823058
:101B300011F1843049F586EE0E94101686EE0E945F
:101B4000E31688E10E94101688E11CC082EE0E9414
:101B500010161AC080EE0E94101681EE0E94101618
:101B600088E10E94101688E10E94E31681EE0E942F
:101B7000E31680EE07C082EE0E94101687E50E94F1
:101B8000101687E50E94E3168FE39CE90197F1F7B1
:101B900000C00000089580915302813029F010F0B8
:101BA000823041F482EE04C08CE20E9410168CE276
:101BB0000E94E31680915D0381FF03C081EE0E94C5
:101BC000101680915D0385FF03C085EE0E941016FC
:101BD00080915D0380FF03C080EE0E94101680910B
:101BE0005D0384FF03C084EE0E94101680915D03A4
:101BF00082FF03C082EE0E94101680915D0386FF73
:101C000003C086EE0E94101680915D0383FF03C01F
:101C100083EE0E94101680915D0387FF03C087EE5C
:101C20000C9410160895EF92FF921F93CF93DF93B9
:101C30007C01CCE0D0E097010C2E02C036952795B0
:101C40000A94E2F7122F1F70812F0E94E5090E946B
:101C50001016812F0E94E5090E94E3162497CC3FBD
:101C60008FEFD80741F7DF91CF911F91FF90EF9051
:101C70000895882319F05198599A02C0519A599899
:101C80005098589A95E09A95F1F70000509A589814
:101C900095E09A95F1F70000882311F0519A599830
:101CA00085E08A95F1F7000008958BB18C7F8BB9A0
:101CB0005098589A5198599A85E08A95F1F7000002
:101CC00008958AB18C7F8AB985E08A95F1F7000082
:101CD000519A599885E08A95F1F70000509A5898E2
:101CE00085E08A95F1F7000008955098589A85E0AC
:101CF0008A95F1F700005198599A85E08A95F1F795
:101D000000000895CF93DF93D82FC8E08D2F8078FF
:101D10000E94390EDD0FC150C9F780E00E94390ED4
:101D200085E08A95F1F7000085E08A95F1F70000DB
:101D300080E0DF91CF9108952BB1342F309523238C
:101D40003BB1432B3FB7F894FC01680F791FE617AE
:101D5000F70789F0819198E04BB9000000C087FF38
:101D60002BB9880F000000C000C000C02BB900C014
:101D70009A9591F7ECCF3FBF0895AF92BF92CF9263
:101D8000DF92EF92FF920F931F93CF93DF938C011B
:101D9000EB01CFB6D090BC00F8948091BC008B7F53
:101DA0008093BC000E94550E0E94610E84E80E9440
:101DB000820ECC0FDD1FCC0FDD1F78015801AC0E59
:101DC000BD1EEA14FB0431F0F70181917F010E94EE
:101DD000820EF7CF0E94750ECFBED092BC00579AEC
:101DE00040E8BE01C801DF91CF911F910F91FF9094
:101DF000EF90DF90CF90BF90AF900C949C0EEF923D
:101E0000FF920F931F93CF93DF93E901662309F4A9
:101E10004BC0242F30E0EFEFF0E0E61BF109B901F1
:101E2000E69F9001E79F300DF69F300D1124232F80
:101E30008B01031B11095CE3E52EF12CB7010E9415
:101E4000302FFB01BC01069FC001079F900D169F1C
:101E5000900D1124B7010E94302FE230F105B1F04E
:101E600040F4309779F0319711F5832F242F461BDA
:101E700021C0E430F105A1F068F03597C1F4842F5A
:101E8000861B18C0832F262F230F14C0862F830F85
:101E9000E42F03C0E42FE61B842F432F2E2F0AC00C
:101EA000842F462F430F06C0842F242F03C080E0C9
:101EB00020E040E0E42FF0E0E359F74F4491E22FB7
:101EC000F0E0E359F74F9491E82FF0E0E359F74F32
:101ED000E49149839883EA83DF91CF911F910F9119
:101EE000FF90EF90089588E090E00C94662FAB018E
:101EF000BC0188E090E00C94842FEEE5F3E083E0F1
:101F0000808310925F038FEF8283838360915E03EF
:101F100070915F0380916003909161030C94770F3F
:101F200080915E0380FF06C06FE070E086E693E07C
:101F30000C94BD0E80E090E0FC01EA59FC4F118248
:101F40001082128204968C339105B1F7EDCF20E018
:101F500030E0F901EA59FC4F8183608342832C5FB2
:101F60003F4F2C333105A9F70C94900FEF92FF925D
:101F70000F931F93CF93DF9300D000D0CDB7DEB780
:101F800000915E0310915F03209160033091610323
:101F900000936203109363032093640330936503FB
:101FA00020915E0320FF21C0042FF62EE92E182F6A
:101FB0009E012F5F3F4F0E94FF0E8091620310FB36
:101FC00087F9809362031695809163038078182BBC
:101FD000E0FA17F910936303F0926403009365032A
:101FE0004B8169818A810E94A70F0F900F900F90FB
:101FF0000F90DF91CF911F910F91FF90EF90089577
:102000008F929F92AF92BF92CF92DF92EF92FF9208
:102010000F931F93CF93DF93EC01062F142F809122
:102020005E0380FF8CC0982F9E77923021F4CE0102
:102030000E94B60F5AC0E82FE695EF739EE39E0FFD
:102040009F73943018F4109161034FC09AE39E0F70
:102050009F73993070F4881F8827881F90915F03C1
:10206000292F220FC22FC82B97FB992790F9D92F20
:102070003CC087E28E0F8F738A30B8F5F0E0799715
:10208000E0FD02C021E001C02FEFEE7FEA5AF84FD9
:10209000859194916FE070E00E94302F26036001DB
:1020A000279FD00C11244E0188E9881A8EEF980AD8
:1020B00086E6E82E83E0F82E98E6A92EBB24B3949A
:1020C000C401B5010E94302F9701412F602F0E945B
:1020D000FF0E8C0C9D1C94E0E90EF11C82EAE816C0
:1020E00083E0F80669F70E94900F80915E039C2FB1
:1020F000C0FB87F980935E03969580915F0380789B
:10210000892BD0FB87F980935F03009360031093C2
:10211000610360915E0370915F0380916003909111
:102120006103DF91CF911F910F91FF90EF90DF90AE
:10213000CF90BF90AF909F908F900C94770FDF91CE
:10214000CF911F910F91FF90EF90DF90CF90BF90B4
:10215000AF909F908F900895EEE5F3E02081221FCD
:102160002227221F30915F03432F440F842F822B9D
:1021700037FB992790F90C9668E671E00E94442F8E
:10218000438162810C94001020915E03221F22275C
:10219000221F30915F03432F440F842F822B37FB84
:1021A000992790F98C3091051CF4845A9E4F01C0F8
:1021B0000C9768E671E00E94442F409161036091A2
:1021C00060030C940010EEE5F3E08081881F8827FF
:1021D000881F90915F03292F220F97FB992790F971
:1021E00043816FEF822B0C940010EEE5F3E08081C9
:1021F000881F8827881F90915F03292F220F97FB44
:10220000992790F9438160E0822B0C940010409153
:102210006103842F90E0843F910514F4445F01C072
:102220004FEF80915E03881F8827881F90915F037E
:10223000292F220F97FB992790F960916003822B39
:102240000C94001040916103842F90E00C9714F0DF
:102250004C5001C040E080915E03881F8827881F92
:1022600090915F03292F220F97FB992790F9609196
:102270006003822B0C94001090915E0390FF42C08B
:102280009178811102C0926007C0833210F094648B
:1022900003C08F73880F982B90935E0360915E0349
:1022A00070915F0380916003909161030E94770FAA
:1022B00080915E03982F9E77923019F410926902F4
:1022C00010C0982F96959F732EE3290F2F732731F7
:1022D00020F491E09093690204C0995D9F739A3055
:1022E00068F3881F8827881F90915F03292F220F8A
:1022F00097FB992790F94091610360916003822BCD
:102300000C940010089580912C03816080932C031D
:1023100081E080936A020E945D21811104C00E94C5
:102320003C210E947D0F0E94730F60935E037093A7
:102330005F0380936003909361036E7761F40E9462
:102340007D0F0E94730F60935E0370935F03809311
:1023500060039093610381E08093690280915E0342
:1023600080FF04C086958F730C943C110895809172
:102370005E0386958F738F5F833208F081E00C9443
:102380003C1180915E03982F909590FB80F980938B
:102390005E0360915E0370915F0380916003909192
:1023A00061030E94770F80915E0380FF04C08695D1
:1023B0008F730C943C11109269022FEF80E792E02A
:1023C000215080409040E1F700C000000C94900F35
:1023D000CF93C82F80916702909168020E94FE21DE
:1023E000EC2FF0E0E759F84FE491F0E08E179F07EB
:1023F00018F10E94F2219093680280936702E091A5
:102400006602F0E0E359F84F449180915E03881F23
:102410008827881F90915F03292F220F97FB992708
:1024200090F960916003822B0E94B60F8091660242
:1024300090E0019680936602CF910895CF93C82FC4
:1024400080916402909165020E94FE21EC2FF0E0E1
:10245000EA59F84FE491F0E08E179F07E8F00E94E8
:10246000F221909365028093640240916103609130
:10247000600380916202909163020E94B60F809186
:10248000620290916302019668E671E00E94302F2B
:102490009093630280936202CF910895CF92DF926E
:1024A000FF920F931F93CF93DF93F82E80916002DA
:1024B000909161020E94FE21EF2DE695F0E0EA592D
:1024C000F84FE491F0E08E179F07E8F10E94F221A7
:1024D000909361028093600206E613E0C0E0D0E0D2
:1024E00088E6C82EDD24D39480915E0290915F022D
:1024F0008C0F9D1FB6010E94302F980140916103FF
:10250000609160030E94FF0E68960C5F1F4FC836F3
:1025100081E0D80749F70E94900F20915E02309128
:102520005F02F0FE0AC0C9010196BE010E94302F71
:1025300090935F0280935E0206C021503109309370
:102540005F0220935E02DF91CF911F910F91FF9068
:10255000DF90CF9008958F929F92AF92BF92CF92CB
:10256000DF92EF92FF920F931F93CF93DF93C82FC9
:1025700080FF03C0DD24DA9402C0DD24D39480916F
:102580005C0290915D020E94FE21C695EC2FF0E066
:10259000ED59F84FE491F0E08E179F0708F467C0FB
:1025A0000E94F22190935D0280935C0296E6E92EF0
:1025B00093E0F92E08E613E0C0E0D0E027E0822E99
:1025C000912CF80131971082F7011082F8011082E6
:1025D00087E0A82EB12CC12C80915B028C0D87FD69
:1025E000815F082E000C990BC817D907E9F42091D8
:1025F00061032A9DC0012B9D900D1124B4010E94FE
:10260000442F462F80915E03881F8827881F909152
:102610005F03592F550F97FB992790F99701609108
:102620006003852B0E94FF0ECD0CF1E0AF1AB108BC
:1026300099F6219684E0E80EF11C0C5F1F4FCF3015
:10264000D10509F0BECF0E94900F80915B0291E00E
:10265000D91206C0811102C08EE007C0815005C0AA
:1026600090E00196BE010E94442F80935B02DF91AF
:10267000CF911F910F91FF90EF90DF90CF90BF907F
:10268000AF909F908F9008959F92AF92BF92CF92FC
:10269000DF92EF92FF920F931F93CF93DF93CDB70B
:1026A000DEB7EC970FB6F894DEBF0FBECDBF182F84
:1026B0008091590290915A020E94FE21E12FF0E090
:1026C000E05AF84FE491F0E08E179F0708F495C0A8
:1026D0000E94F22190935A0280935902CE010196F2
:1026E0007C015E0193E0A90EB11CC12CD12C8701A5
:1026F000F50131971082F7011082F5011082912CBB
:102700009091010180915802999E800D112487FDBE
:1027100004C08F301CF08EE001C080E0082E000C59
:10272000990BC816D906A1F480915E03881F8827EB
:10273000881F90915F03592F550F97FB992790F9A8
:1027400097014091610360916003852B0E94FF0E09
:102750009394F7E09F12D4CF8FEFC81AD80A94E071
:10276000E90EF11CE4E0AE0EB11CFFE0CF16D1047F
:1027700009F0BECF28E633E099E0E92EF12C4FE0D6
:10278000C42ED12CC701B6010E94442FD901119744
:10279000FC01EE0FFF1FEE0FFF1FE00FF11F818105
:1027A0008C93119780818C938281F9018083FFEF54
:1027B000EF1AFF0A2C5F3F4F88E1E816F10411F78A
:1027C0000E94900F9091010180915802913049F43C
:1027D0008A3F2CF489EF809358028FEF08C0815014
:1027E0000AC086313CF085E18093580281E08093F5
:1027F000010103C08F5F80935802EC960FB6F894E6
:10280000DEBF0FBECDBFDF91CF911F910F91FF9023
:10281000EF90DF90CF90BF90AF909F900895EF9290
:10282000FF920F931F93CF93DF9380915602909165
:1028300057020E94FE21883E9340D0F10E94F2216F
:102840009093570280935602C0915402D091550242
:102850002196C170DD27D0935502C093540286E6BD
:10286000E82E83E0F82E10E008E7812F8695FE0120
:10287000E80FF11DCF018170992797014091610305
:1028800060916003FC010E9FC0010F9F900D112409
:102890000E94FF0E1F5FF4E0EF0EF11C1F3029F7BE
:1028A000DF91CF911F910F91FF90EF900C94900FBB
:1028B000DF91CF911F910F91FF90EF90089580913C
:1028C0006902882391F190915E03892F86958F7319
:1028D0002EE3280F2F73243018F482500C94E81143
:1028E0002AE3280F2F73233018F486500C941E12FD
:1028F00027E3280F2F73263018F489500C944E12BA
:1029000021E3280F2F73263018F48F500C94AB124C
:102910002BE2280F2F73233018F485510C944413A5
:102920009E77903311F40C940F14089590937002D5
:1029300080936F020895E0916F02F09170023097DA
:1029400021F00190F081E02D099480E00895E0915C
:102950006F02F0917002309721F00280F381E02D38
:1029600009940895E0916F02F0917002309721F080
:102970000480F581E02D0994089520916D02309135
:102980006E028217930771F090936E0280936D022E
:10299000E0916F02F0917002309721F00680F7818C
:1029A000E02D0994089520916B0230916C028217FA
:1029B000930771F090936C0280936B02E0916F0229
:1029C000F0917002309721F00084F185E02D099498
:1029D000089508950C94E9140E94E9210E94540678
:1029E0000E9470220C948311CF92DF92EF92FF929B
:1029F0000F931F93CF93DF93CDB7DEB72B970FB60F
:102A0000F894DEBF0FBECDBF0E94C00682E7C82E7D
:102A100082E0D82E00E010E0E02E802F0E94A20776
:102A2000F60141916F01F42EF826B1F40F5F1F4FAC
:102A30000E30110589F78FEF89838A831B820E94EC
:102A4000F2218160782F9D838C8349815A816B812B
:102A50008D810E94D31540C090912C0391FF04C03A
:102A60008B870E94A8078B8520E030E04F2D50E037
:102A7000922FBA01022E02C0759567950A94E2F76B
:102A800060FF24C02E83EF8221E030E0690102C0A4
:102A9000CC0CDD1C9A95E2F790E08C219D21892BCE
:102AA00009F420E028870E94F2218160782F9A871C
:102AB00089874E815F8168858A850E94D315F801D8
:102AC000EE58FD4F8081C826C08206C02F5F3F4F61
:102AD0002630310569F6AACF0E94032410917102B5
:102AE0000E949B141817A1F00E949B1480937102FE
:102AF0002B960FB6F894DEBF0FBECDBFDF91CF91FE
:102B00001F910F91FF90EF90DF90CF900C94F509FB
:102B10002B960FB6F894DEBF0FBECDBFDF91CF91DD
:102B20001F910F91FF90EF90DF90CF900895DC01FF
:102B300011962C9111978C91682F70E041E050E034
:102B400001C0440F8A95EAF712968C91129730E0F3
:102B5000882329F080918F028823E9F006C0F901CB
:102B6000E058FD4F90819423B1F086E0829FF00100
:102B7000839FF00D1124E60FF71FEE0FFF1FEC5E91
:102B8000FE4F808191818D939C93F901E058FD4F18
:102B90008081482B06C0F901E058FD4F40958081A7
:102BA000482340830895CF93DF93CDB7DEB72B97AB
:102BB0000FB6F894DEBF0FBECDBF942F4F83252FE5
:102BC000588769877A878B874A855B85452B21F0F3
:102BD0002F3F09F59F3FF9F4DE01119686E0FD01D4
:102BE00011928A95E9F785E0FE01379601900D92E2
:102BF0008A95E1F749815A816B817C818D819E8123
:102C00000E94C61C2B960FB6F894DEBF0FBECDBF38
:102C1000DF91CF910895CE0107960E949715DCCFE2
:102C2000CF93882309F4CDC0C82F823859F40E946D
:102C30009B1481FDC6C089E30E94ED1F0E94BD2048
:102C400089E30CC0833879F40E949B1480FDB9C0DD
:102C500083E50E94ED1F0E94BD2083E50E942F2086
:102C6000CF910C94BD20843859F40E949B1482FDAE
:102C7000A8C087E40E94ED1F0E94BD2087E4EECF2C
:102C80008CEF8C0F813A48F48C2F0E9443268111DF
:102C900098C08C2F0E94ED1FE3CF80E28C0F88300C
:102CA00048F4C77081E001C0880FCA95EAF70E9416
:102CB0007620D6CF8BE58C0F833078F4C53A29F097
:102CC000C63A31F083E890E005C081E890E002C0A8
:102CD00082E890E0CF910C94BD1488E58C0F85318B
:102CE00008F06FC0C83A61F1C93A69F1CA3A71F1A6
:102CF000CB3A79F1CC3A81F1CB3B89F1CC3B91F1E4
:102D0000CD3A99F1C03BA1F1CE3AA9F1CF3AB1F158
:102D1000C13BB9F1C23BC1F1C33BC9F1C43BD1F1E5
:102D2000C53BD9F1C63BE1F1C73BE9F1C83BF1F145
:102D3000C93BF9F1CA3B09F43FC080E090E03EC0D6
:102D400082EE90E03BC089EE90E038C08AEE90E0E1
:102D500035C085EB90E032C086EB90E02FC083EB6E
:102D600090E02CC084EB90E029C087EB90E026C077
:102D70008CEC90E023C08DEC90E020C083E891E0E3
:102D80001DC08AE891E01AC082E991E017C084E989
:102D900091E014C081E292E011C083E292E00EC0A3
:102DA00084E292E00BC085E292E008C086E292E005
:102DB00005C087E292E002C08AE292E0CF910C94D3
:102DC000D314CF910895882309F44BC0823859F465
:102DD0000E949B1481FF45C089E30E94ED1F0E9461
:102DE000BD2089E30CC0833871F40E949B1480FFDE
:102DF00038C083E50E94ED1F0E94BD2083E50E943C
:102E00002F200C94BD20843859F40E949B1482FF1B
:102E100028C087E40E94ED1F0E94BD2087E4EFCF09
:102E20009CEF980F913A58F390E2980F983050F435
:102E3000877091E001C0990F8A95EAF7892F0E9467
:102E40007C20DFCF9BE5980F933020F480E090E06A
:102E50000C94BD14885A853120F480E090E00C94E5
:102E6000D3140895882321F00E9476200C94BD206D
:102E70000895882321F00E947C200C94BD200895A1
:102E80008F929F92AF92BF92CF92DF92EF92FF927A
:102E90000F931F93CF93DF931F92CDB7DEB77C01C3
:102EA000C72EFC01058102950F701281112321F0BC
:102EB00069830E949320698169830E94E61F69816A
:102EC000882381F0112371F080E2860F883050F062
:102ED00082E00E94CF1F0E94E61F91E0D82ED926E3
:102EE000698101C0D12CAC2CA2948FE0A822B12C16
:102EF000F501E159FF4F0C94582F8C2D807F0C2D3C
:102F00000F70882311F00295007F1123C1F0002378
:102F100009F4D2C180E2860F883010F0611105C03B
:102F2000802F69830E94762004C0802F69830E94CD
:102F30008620698169830E94BD206981BDC1862F79
:102F400069830E94E3166981002309F40EC280E2BE
:102F5000860F883010F0611104C0802F0E947C2001
:102F600003C0802F0E948C200E94BD20FEC19C2D9A
:102F7000907F8C2D8F70903211F08295807F662328
:102F800019F06130B1F01EC0112349F0002309F49B
:102F90004BC1013009F048C10E94A620E6C10023C0
:102FA00019F0013009F4E1C189830E94A9208981C7
:102FB00041C1112321F0023008F0D7C135C1011100
:102FC000D4C138C1112321F0002309F42DC174C1EB
:102FD000002309F42FC181C18C2D869586958370BD
:102FE00090E0009719F0019761F0BFC1112321F023
:102FF000862F9C2D937002C080E090E00E94BD144B
:10300000C4C1112321F0862F9C2D937002C080E053
:1030100090E00E94D314B9C11123F9F0653F51F03B
:10302000663F71F0643FA9F48091A2039091A303DD
:1030300081600BC08091A2039091A303826005C0C0
:103040008091A2039091A30384609093A303809343
:10305000A203862F0E940B231EC0653F51F0663FDE
:1030600071F0643FA9F48091A2039091A3038E7F35
:103070000BC08091A2039091A3038D7F05C0809126
:10308000A2039091A3038B7F9093A3038093A20349
:10309000862F0E9473230E94F82377C18C2D8370A2
:1030A00009F052C011116DC1862F829586958770E7
:1030B000880F880F962F9F70892E912CA12CB12CF0
:1030C000082E04C0880C991CAA1CBB1C0A94D2F7B9
:1030D00064FF14C00FE010E020E030E0B901A80167
:1030E00004C0440F551F661F771F8A95D2F7CB0186
:1030F000BA01609570958095909503C060E070E08E
:10310000CB012C2D26952695237030E022303105F9
:1031100069F02330310589F0682979298A299B29AA
:103120002130310571F00E94091E2BC168297929CF
:103130008A299B290E941B1E24C10E94091EC501C9
:10314000B4010E94F71D1DC1112319F08C2D81704F
:1031500001C08695882309F414C1862F829586952F
:103160008770880F880F962F9F70892E912CA12C25
:10317000B12C082E04C0880C991CAA1CBB1C0A94F4
:10318000D2F764FF14C00FE010E020E030E0B90196
:10319000A80104C0440F551F661F771F8A95D2F7F8
:1031A000CB01BA01609570958095909503C060E061
:1031B00070E0CB012C2D269526952370422F50E0F0
:1031C0004230510569F04330510589F06829792969
:1031D0008A299B294130510571F00E94CD1ED1C032
:1031E000682979298A299B290E94DF1ECAC00E946A
:1031F000CD1EC501B4010E94BB1EC3C0862F90E046
:10320000FC01E05EF109E531F10508F051C0E1583B
:10321000FF4F0C94582F062F0F708C2D8F71112398
:1032200031F00E94541E802F0E9432179EC00E94CF
:10323000751E802F0E94391798C0112339F0011193
:1032400094C08C2D8F710E949A1E8FC0023008F09E
:103250008CC0F7CF112339F08C2D8F710E94541E32
:1032600084C01123C9F38C2D8F710E94751E7DC0FF
:10327000112329F08C2D8F710E943F1E76C00E9471
:103280003A1E73C0112351F01C2D1F71812F0E9413
:10329000541E63E0812F0E94C61F67C081E00E9418
:1032A000CF1F023008F461C082E00E94CF1F5DC0D2
:1032B000112331F0002381F2862F0E94101655C091
:1032C000002389F2693349F45FEF77EE83E05150D0
:1032D00070408040E1F700C00000862F0E94E31696
:1032E00044C04C2D4F70C7010E94A9070E946A1D5F
:1032F0004CC0623F99F128F4603F49F0613FE1F032
:1033000020C0643FA1F050F0653F59F01AC011236E
:1033100039F190918F0281E0892706C081E018275A
:103320001DC011111DC081E080938F0219C01111C1
:1033300017C010928F0214C0002381F0111110C029
:10334000E8CF002359F0862F6983112319F00E94DA
:10335000101602C00E94E316698102C010938F020A
:103360004C2D4F70C7010E94F70998E0A916B104CF
:1033700041F05CF0FAE0AF1AB10822E0A216B10405
:1033800020F40E949B140E94F509DD20F1F00E94B8
:10339000C21F80FD1AC0F70112820E94BC1F0E944A
:1033A000541EC7010E94F3190E94BC1F0F90DF91A9
:1033B000CF911F910F91FF90EF90DF90CF90BF9032
:1033C000AF909F908F900C94751E0F90DF91CF91CE
:1033D0001F910F91FF90EF90DF90CF90BF90AF9033
:1033E0009F908F9008950F931F93CF93DF93EC01DD
:1033F000888199812B813C81232BB9F09F3F11F467
:103400008F3F99F0CE010E941908882371F06881DE
:1034100079818A810E94991F8C010E94F11E0E946D
:10342000F41DB801CE010E944017DF91CF911F918A
:103430000F9108950E9493200E94A3200E9465206E
:103440000E94BD200E94A8240E94F82380E090E002
:103450000E94BD1480E090E00C94D3140E9483205D
:103460000C941A1A0E948E1FE92FE295EF70F0E07B
:103470003297EE30F105B0F4EC56FF4F0C94582F14
:10348000803F91F018F4803E68F40EC0843F51F400
:103490000BC0803E48F0813F29F406C093FB88278B
:1034A00080F9089580E0089581E00895CF93DF9337
:1034B00000D000D01F92CDB7DEB70F900F900F90C5
:1034C0000F900F90DF91CF910895CF93DF9300D0AD
:1034D00000D000D0CDB7DEB726960FB6F894DEBF89
:1034E0000FBECDBFDF91CF9108951F93CF93DF9390
:1034F000C091900216E080919102C81799F0D0E037
:103500001C9FF0011D9FF00D1124EE56FD4F4081D0
:10351000518162817381848195810E94651A21960F
:10352000C770E9CFDF91CF911F9108954091C202FA
:103530005091C3026091C4027091C5028091C6028D
:103540009091C7020C94651A8091C70282958F7082
:1035500009F054C08091C402882309F44FC08091BF
:103560009002A09191026091C2027091C3024091B9
:10357000C5025091C602B6E08A1709F43FC090E038
:1035800041155105C1F17F3F11F46F3FA1F1B89F83
:10359000F001B99FF00D1124EE56FD4F21817213F9
:1035A0002AC02081621327C02281211124C02381D7
:1035B00034812417350710F421503109241B350BB1
:1035C000283C3105C0F42091C7022F702061209360
:1035D000C70226E0289FF001299FF00D1124E9562B
:1035E000FD4F80818F708061808382EC92E00E9429
:1035F000F3190C94751A01968770BECF0895CF9277
:10360000DF92EF92FF920F931F93CF93DF93CDB78B
:10361000DEB762970FB6F894DEBF0FBECDBF8C0148
:1036200085E0F801DE011D9601900D928A95E1F783
:10363000D8014C9111965C91119712966C9112974A
:103640001396CD90DC9014973091C2027091C30212
:103650008091C5029091C602009709F46BC17F3F2B
:1036600019F43F3F09F466C1E090C402EE2009F46A
:10367000C0C02091C702C816D90628F0F601E81B81
:10368000F90BCF0104C0809590958C0D9D1DFF24F2
:10369000F394883C910578F0F12C207F09F0C6C0A6
:1036A0007C2DD98AC88A89890E94561A82EC92E0B8
:1036B0000E94F319B1C0822F807F09F046C07513B4
:1036C00014C0341312C0611110C02F7020612093F8
:1036D000C7020E94961A82EC92E00E94F319809130
:1036E000C702D80115968C932EC0CD2819F15F3FE3
:1036F00011F44F3FF9F0F62E61111CC08091900239
:103700002091910236E0821709F45AC090E0389F68
:10371000F001399FF00D1124EE56FD4F71815713C2
:1037200006C07081471303C07281711103C00196F6
:103730008770E9CFF62E662309F418C18091C7027D
:1037400081608093C702F12C11C1751308C0341336
:1037500006C0611104C08091C702D801C3C04D8763
:103760005E878D859E856A8B0E94321A6A898823BE
:10377000E1F16623D1F12091C702822F82958F70EB
:1037800090E0029774F08091C2029091C3029887F2
:103790008F831986DB86CA862C87CE0107960E9406
:1037A000F31986E0F801A2ECB2E001900D928A953F
:1037B000E1F70E94A41A0E94961AFF24F394D6C03F
:1037C0004D875E878D859E850E948E1F292F2295AD
:1037D0002F7030E0223031050CF0BCC09F7009F032
:1037E000B6C0805E883008F4C1C0C8010E94F319D9
:1037F000E4CFC816D90608F453C0F601E81BF90B4C
:10380000CF01883C910508F450C0F12C7C2DD98A59
:10381000C88A89890E94561AE2ECF2E086E0DF014C
:103820001D928A95E9F70E94961AA0C0751314C0DC
:10383000341312C0611110C08091C702F801858352
:10384000C8010E94F31986E0E2ECF2E0DF011D926C
:103850008A95E9F7FE2C8AC04D875E878D859E8507
:103860006A8B0E94321A6A89882309F4BECF6623C4
:1038700009F4BBCF2091C702822F82958F7090E010
:1038800002970CF48ECF8091C2029091C3029A836A
:1038900089831B82DD82CC822E83CE0101967FCF6D
:1038A000809590958C0D9D1DACCFF62E662309F466
:1038B0009CCF75132EC034132CC02091C70220FD5D
:1038C0001FC0822F82958F70D9F0D80115962C9346
:1038D00015978F3049F08F5F982F9295907F822FA8
:1038E0008F70892B15968C93C8010E94F31986E07E
:1038F000F801A2ECB2E001900D928A95E1F793CF26
:1039000086E0F801A2ECB2E001900D928A95E1F711
:103910002DC04D875E878D859E850E94321A81114C
:1039200040CF8091C70281608093C702C8010E9486
:10393000F3191CC0662309F458CF4D875E878D8527
:103940009E850E94321A882309F44FCF2ACF811115
:1039500048CF0CC0243031050CF047CF9F7009F4DC
:1039600040CFF8019581907F09F03BCF8F2D629673
:103970000FB6F894DEBF0FBECDBFDF91CF911F9180
:103980000F91FF90EF90DF90CF9008951F93CF930A
:10399000DF93CDB7DEB72C970FB6F894DEBF0FBE1E
:1039A000CDBF4F83588769877A878B879C87CE01E5
:1039B00007960E94FF1A882369F08F8198852A85CF
:1039C0003B85232BF1F19F3F09F063C08F3F09F046
:1039D00060C037C086E0FE013796DE011196019087
:1039E0000D928A95E1F76F817885EA85FB8530979E
:1039F00041F17F3F11F46F3F21F12091910230E0BE
:103A0000C9010196877099274091900250E0841770
:103A1000950709F447C069837A83FD83EC8396E0B8
:103A2000929FD001939FB00D1124AE56BD4FFE0161
:103A3000319601900D929A95E1F7809391020E9440
:103A4000751A16E080919002909191028917C1F148
:103A5000189FC00111248E569D4F0E94FF1A882383
:103A600079F1E09190021E9FF0011124EE56FD4F76
:103A70004081518162817381848195810E94651AA0
:103A80008091900290E00196877099278093900230
:103A9000D9CF4F81588569857A858B859C850E9411
:103AA000651ACFCF0E942E1A1092910210929002A6
:103AB000E2ECF2E086E0DF011D928A95E9F7C1CFE2
:103AC0002C960FB6F894DEBF0FBECDBFDF91CF911D
:103AD0001F910895EF92FF920F931F93CF93DF935F
:103AE0008C01892B09F46CC0F12CEE24E394E801DD
:103AF0002196F8018491843740F4843008F051C055
:103B0000813081F0823019F15BC0853709F444C0FF
:103B1000A8F19CE7980F903708F052C08F770E9469
:103B2000E31641C00E5F1F4FFE01C49180E28C0F6F
:103B3000883048F4C7708E2D01C0880FCA95EAF707
:103B40000E94962014C08C2F0E9410162DC00E5F6C
:103B50001F4FFE01C49180E28C0F883058F4C7706B
:103B60008E2D01C0880FCA95EAF70E949C200E9402
:103B7000BD201AC08C2F0E94E31616C00E5F1F4F87
:103B8000FE01C491CC2381F08FE99FE00197F1F70A
:103B900000C00000C150F6CF0E5F1F4FFE01F49031
:103BA00003C00E9410168E018F2D882309F49FCF29
:103BB000EFE9FFE03197F1F700C000008150F5CF49
:103BC000DF91CF911F910F91FF90EF90089508958D
:103BD0000E94E71D60930303709304038093050321
:103BE000909306030C941A1A08950C94E81D0F93F1
:103BF0001F9300910303109104032091050330915A
:103C00000603602B712B822B932B1F910F910C9429
:103C1000E81D0F931F93009103031091040320915B
:103C200005033091060360237123822393231F91A0
:103C30000F910C94E81D0F931F93009103031091B3
:103C40000403209105033091060360277127822722
:103C500093271F910F910C94E81D08950E942D1E2B
:103C60006093FF027093000380930103909302031B
:103C70000C941A1A60E070E0CB010C942E1E0F9386
:103C80001F9341E050E060E070E08A019B0104C0B6
:103C9000000F111F221F331F8A95D2F7C901B801E7
:103CA0001F910F910C942E1E0F931F9341E050E033
:103CB00060E070E004C0440F551F661F771F8A95AF
:103CC000D2F78091FF0290910003A0910103B0917F
:103CD00002038A019B01082B192B2A2B3B2BC901BC
:103CE000B8011F910F910C942E1E0F931F9341E06A
:103CF00050E060E070E004C0440F551F661F771F5E
:103D00008A95D2F740955095609570958091FF0205
:103D100090910003A0910103B09102038A019B01DD
:103D2000082319232A233B23C901B8011F910F91AE
:103D30000C942E1E0F931F9341E050E060E070E062
:103D400004C0440F551F661F771F8A95D2F78091D4
:103D5000FF0290910003A0910103B09102038A0138
:103D60009B01082719272A273B27C901B8011F9162
:103D70000F910C942E1E0F931F930091FF02109130
:103D800000032091010330910203602B712B822BE1
:103D9000932B1F910F910C942E1E0F931F93009144
:103DA000FF02109100032091010330910203602370
:103DB0007123822393231F910F910C942E1E0F9336
:103DC0001F930091FF021091000320910103309195
:103DD000020360277127822793271F910F910C946C
:103DE0002E1E0895292F220F920F990F890FA82FA9
:103DF000A695A695A695877051E001C0550F8A95A6
:103E0000EAF785E0A89FD001112420E030E070E0BF
:103E1000F901EA0FFB1FE853FD4F4081CB01022E51
:103E200002C0969587950A94E2F78170992781954B
:103E300084278523842780832F5F3F4F25303105DA
:103E400039F70895292F220F920F990F890F682FA4
:103E5000669566956695982F977085E0689FB00186
:103E6000112440E050E080E0FA01E60FF71FE8532C
:103E7000FD4F208130E0092E02C0369527950A9427
